:020000040800F2
:10000000F8FF01206D4805088FB904087DB9040880
:1000100091B90408A1B90408B1B9040800000000AE
:10002000000000000000000000000000C1B904084A
:10003000C3B904080000000039CA040895CA0408BE
:1000400063470508B1BA0408BDBA0408C5BA040874
:10005000C53805086347050845BA04084BBA0408C3
:1000600051BA040857BA04085DBA040879EC0408C8
:1000700089EC040899EC0408A9EC0408B9EC04081C
:10008000C9EC0408D9EC0408634705080000000027
:1000900000000000000000000000000063BA040837
:1000A000D9BA0408DFBA0408F1BA0408F7BA040898
:1000B000FDBA040803BB040809BB04083BBB0408E1
:1000C00041BB040847BB04084DBB0408634705084F
:1000D0006347050829BB04082FBB04080000000083
:1000E00087BA0408B7BA0408D1B9040800000000B0
:1000F000000000000000000000000000E9EC04081F
:10010000000000006347050811BB040863470508A9
:1001100000000000000000000000000000000000DF
:10012000F9EC040809ED040819ED040829ED0408A8
:1001300039ED04080000000000000000000000008D
:10014000000000000000000000000000C5B9040825
:1001500049ED040859ED040869ED040835BB0408AD
:1001600053BB040859BB0408000000000000000055
:10017000000000000000000000000000000000007F
:1001800000000000634705080000000000000000B8
:10019000634705086347050842884378007843EAC7
:1001A000022340EA032070470B0A017043700B0CD6
:1001B000090E8370C1707047036A0239023B8B429B
:1001C00083BFC389406B01FB03000020704700F12F
:1001D0000B010022D30143EA520310F8012B52FA1B
:1001E00083F38842DAB2F5D11046704737B50D4631
:1001F000044620B9092000232B6003B030BD0368FA
:10020000002BF7D05A79002AF4D081885A8991427C
:10021000F0D118680DF10702062102F0F3FA9DF8FB
:10022000073003F00103034313F0FF00E2D123681A
:10023000E2E738B50568044615F8010B20B140F235
:10024000B51154F06FFB08B1256038BD4FF0FF3099
:10025000FBE7CA7E8B7E032843EA022301BF487D69
:100260000A7D42EA002243EA024318467047C2F37D
:1002700007238A76CB760378032B01BF120C0A750D
:10028000120A4A75704737B5C37904461BB9002571
:10029000284603B030BD00F13C01826B006801913B
:1002A000012302F09AFA054680B9E36AE071A06B77
:1002B000626AC31A9342EAD2A3790199022BE6D16A
:1002C00002440123206802F088FAE1E70125DFE714
:1002D00038B5836B8B4205460C4610D0FFF7D3FF31
:1002E00060B922462868012305F13C0102F066FA54
:1002F00000281CBF4FF0FF340120AC6338BD002044
:10030000FCE7000038B50023C3714FF0FF3383636F
:100310000546FFF7DDFF044618BB95F83B2295F82C
:100320003A3243EA02234AF6552293421BD195F80A
:100330003C30EB2B03D01833DBB2012B15D80C4922
:10034000032205F172003FF0B7FF40B109490522D1
:1003500005F18E003FF0B0FF002818BF02242046B0
:1003600038BD0424FBE70324F9E70224F7E700BFC4
:1003700002E8060806E806082DE9F047437986B04A
:10038000044601F0FE0593B10DF107020068062155
:1003900002F038FA9DF80730DA0708D41DB113F0DF
:1003A000040500D00A25284606B0BDE8F0870023E2
:1003B000637120680DF10702052102F023FA9DF810
:1003C000073013F0010840F014810DB15B07E9D448
:1003D00000212046FFF796FF022803D0012823D8EA
:1003E000277987B302AD04F2022104F242272E4698
:1003F00011F8040C10B10846FFF7CEFE10318F4201
:1004000045F8040BF4D1257905B1013D56F8257066
:100410007FB139462046FFF775FF23795BB9012884
:1004200011D90135032DF1D9042808D14FF0010865
:1004300007E00320F1E70428F8D0012803D94FF0A2
:100440000D084546AFE794F8482094F8473043EA52
:100450000223B3F5007FF2D194F8530094F8526070
:1004600056EA002604D104F16000FFF795FE064627
:1004700094F84C5066626B1E012BA571DFD894F87E
:100480004990A4F80E904B46002BD8D009F1FF33C9
:1004900013EA090FD3D194F84E3094F84DA04AEAEC
:1004A000032A1AF00F0F0FFA8AF1A4F80CA0C6D194
:1004B00094F8503094F84F0050EA032003D104F12F
:1004C0005C00FFF769FE94F84BE094F84A3053EA79
:1004D0000E2EB4D006FB05FC0EEB1A1262448242CB
:1004E000ADD8801A4845B0FBF9F5A8D3464B9D42DC
:1004F000A5D84FF6F5739D427DD94FF0030902351B
:100500000EEB07033A44B9F1030F2562A762E362D9
:1005100062635CD194F8672094F8663043EA022362
:100520000B431BB2002B8AD104F16800FFF734FEA5
:10053000AD00206305F2FF15B6EB552FFFF47FAF3A
:100540004FF0FF33C4E90533B9F1030F4FF08003D7
:1005500023722FD194F86D2094F86C3043EA022373
:10056000012B27D1791C2046FFF7B2FE10BB94F86F
:100570003B2294F83A32207243EA02234AF655228B
:10058000934217D104F13C00FFF706FE1F4B98423F
:1005900010D104F50870FFF7FFFD1D4B984209D1FB
:1005A00004F50970FFF7F8FDA06104F50A70FFF784
:1005B000F3FD6061174A84F80590138801339BB2FC
:1005C00013806381144B23610023E36139E7BAF19F
:1005D000000F3FF434AF6344B9F1020F23634FEAD5
:1005E00045031BBF5B1905F001051D4605EB5305CF
:1005F000A0E70325D7E640F6F5794D458CBF4FF0CF
:1006000002094FF001097AE7F5FFFF0F52526141ED
:10061000727241611C5A00201E5A002001292DE9E6
:10062000F04706460C46174673D9036A8B4270D9C9
:100630004379022B3FD0032B50D0012B69D101EB22
:100640005108C16A01EB5821FFF742FE054638BB4D
:1006500006F13C0908F1010AC8F3080814F0010486
:100660001FBF19F8083003F00F023B0103F0F0033D
:1006700014BF1343FBB209F80830F16A0123F37188
:1006800001EB5A213046FFF723FE054640B9CAF375
:10069000080A44B1C7F3071709F80A700123F37178
:1006A0002846BDE8F08719F80A30C7F3032723F07E
:1006B0000F031F43F0E7C16A01EB1421FFF708FEA7
:1006C00005460028ECD1640006F13C0304F4FF74F5
:1006D00018191F55C7F307274770DFE7C16A01EBF9
:1006E000D411FFF7F5FD05460028D9D1A40006F185
:1006F0003C0304F4FE741C442046FFF74DFD27F034
:10070000704700F0704047EA00012046FFF74CFDBB
:10071000C4E70225C4E70129F8B505460C4652D9BD
:10072000036A99424FD24379022B29D0032B38D048
:10073000012B48D101EB5106C16A01EB5621FFF7AD
:10074000C7FD10B14FF0FF30F8BD771CE96AC6F362
:1007500008062E4401EB5721284696F83C60FFF727
:10076000B7FD0028EED1C7F308073D44E30795F82D
:100770003C0046EA00204CBF0009C0F30B00E3E751
:10078000C16A01EB1421FFF7A3FD0028DAD1640050
:100790003C3504F4FF742B19285D5B7840EA032094
:1007A000D2E7C16A01EBD411FFF792FD0028C9D14D
:1007B000A40005F13C0004F4FE742044FFF7ECFCB7
:1007C00020F07040C0E70120BEE7B1F5001FF8B58A
:1007D00006460C4601D30220F8BDCA06FBD182684A
:1007E00005680161CAB96B79022B01D92B6B9BB9E2
:1007F000AB89B3EB541FEED92B6BB361B369726154
:10080000002BE8D003EB54233C35C4F308042C44FC
:10081000B361F4610020DFE71A46EF897F02BC4232
:10082000114604D22846FFF7C7FCB061E6E73068FE
:10083000FFF771FF431C024606D00128CBD92B6A73
:100840008342C8D9E41BEAE70120C5E72DE9F0415E
:10085000056880460F4649B96E69C6B12B6AB34236
:1008600098BF0126AB69A3B9002406E02846FFF72C
:1008700052FF0128044603D801242046BDE8F08138
:10088000421C51D02B6A8342F7D83E46EAE7012644
:10089000E8E7BE4215D12B6AD8F80000741CA342C9
:1008A00098BF02242146FFF736FF0128E4D0431CFD
:1008B0003AD0D8B16B69012B03D92A6A934238BF69
:1008C0001E4634462B6A0134A34202D8012ECBD9EE
:1008D0000224D8F800002146FFF71DFF40B101288F
:1008E000CAD0013020D0B442ECD1BDE7002CE8D012
:1008F0004FF0FF3221462846FFF790FE90B957B9D6
:100900002A6AAB696C61023A934210D92B7A43F0A0
:1009100001032B72B1E7224639462846FFF77EFED7
:100920000028EDD00128A7D14FF0FF34A5E7013B07
:10093000AB61EBE773B50C46012C05680646114622
:100940002CD92B6AA34229D92AB14FF0FF3228466D
:10095000FFF764FE40B9214630680194FFF7DBFEE3
:100960000199044610B9002002B070BD012815D0CD
:10097000431C15D000222846FFF750FE0028F3D173
:100980002A6AAB69911E8B4205D20133AB612B7A87
:1009900043F001032B72A242DDD8E4E70220E3E733
:1009A0000120E1E7F7B505460191FFF76CFC04462D
:1009B00000BB01992846FFF7FFFB05F13C070646FF
:1009C000A8634FF40072214638463FF05FFCEB8984
:1009D0009C4205D3E889001B18BF012003B0F0BD7D
:1009E000286801233219394601F0F7FE0028F1D1B9
:1009F0000134ECE70120F1E72DE9F84307690668C7
:100A00002037B7F5001F24BF0023836183690446A4
:100A1000894673B1C7F30808B8F1000F39D14169AD
:100A20000133836139B9B389B3EB571F31D8002340
:100A3000A36104200BE0F389013B13EA572328D17B
:100A40003046FFF768FE0128054602D80220BDE8BF
:100A5000F883421C01D10120F9E7336A834212D89E
:100A6000B9F1000FE3D061692046FFF7EFFE0546BC
:100A7000A8B10128EAD0431CEDD001463046FFF76B
:100A800091FF0028E7D1656129463046FFF794FBC6
:100A9000A0613C3646442761E6610020D7E7072085
:100AA000D5E7F8B50E46002107680446FFF78DFE2E
:100AB000A8B90546A1693846FFF70AFC78B9E36989
:100AC0001B78E52B00D01BB90135B54201D1F8BD2B
:100AD000054601212046FFF78FFF0028EAD00428B1
:100AE00008BF0720F3E700002DE9F84FFF27D0F8F3
:100AF0000090064688463D4604244FF6FF7AB169C9
:100B000011B9002C73D063E04846FFF7E1FB0446BF
:100B100000285DD1F0690378002B70D0C27AE52BF4
:100B200002F03F02B27158D02E2B56D022F0200195
:100B3000A1F1080CDCF1000141EB0C0141454CD165
:100B40000F2A4FD15C0646D53269477BF26203F02B
:100B5000BF03427BBA4240D1C17E827E42EA01227B
:100B600011B2002A39D10278D9F81050DFF894E098
:100B700022F04002013A0D2462434FF0010C1EF8AE
:100B8000014B00EB040B045D9BF801B044EA0B241D
:100B9000BCF1000F23D0FF2A1FD825F81240A4462D
:100BA000013201310D29EAD10178490607D5BCF19E
:100BB000000F04D0FF2A10D8002125F812105D1E66
:100BC000EDB200213046FFF717FF0446002896D00B
:100BD0000023B3610CE09D42BBD0FF25F1E75445F3
:100BE000DFD0FAE73DB9FFF7F2FAB84203D10024AB
:100BF0002046BDE8F88F4FF0FF33F362F8E7042496
:100C0000E6E700BFD0E80608C16A4B1C2DE9F041B9
:100C100005680669044618D1E5274FF00108A16967
:100C20002846FFF755FB60B9E3691F7085F8078018
:100C30002369B3420DD201462046FFF7DDFE0028AE
:100C4000EDD0042808BF022003E0FFF7BEFD002816
:100C5000E2D0BDE8F08100002DE9F04F002185B021
:100C6000D0F800A00446FFF7B0FD0746002840F08A
:100C700092804FF0FF334FF0FF09E362C8460093C4
:100C8000A1695046FFF724FB0746002840F0838007
:100C9000E5692E78002E00F08280EA7AE52E02F0D7
:100CA0003F03A37103D0100704D50F2B04D0009B82
:100CB000E36253E00F2B59D194F82B30590643D4FB
:100CC000720649D5236995F80D90E36206F0BF06D8
:100CD0006B7B4B4542D1EA7EAB7E53EA02233DD18A
:100CE0002F78DAF810B007F03F077B1E0D275F431F
:100CF0002C4B012213F8011B681815F8018040786D
:100D000048EA00286AB3FF2F039327D8404653F0E0
:100D10001DFE791C02903BF81700019153F016FE5E
:100D2000029A82421AD10199039B42460F461E49FC
:100D30009942DFD12B785B0603D512B13BF817300F
:100D400063B9013E5FFA86F800212046FFF754FEA2
:100D50000746002894D01EE0B045B9D04FF0FF08F8
:100D6000F2E74FF6FF718845E1D0F7E7B8F1000FE1
:100D700004D12846FFF72BFA48450CD094F82B7085
:100D800017F0010793D10B2204F1200128463FF010
:100D900093FA00288BD1384605B0BDE8F08F0427C0
:100DA000F9E700BFD0E80608DDE806082DE9F04FB6
:100DB00090F82BB01BF0A00489B0054640F0E3800A
:100DC00007683A6932F81430002B6CD105F120061F
:100DD00096E807000DF1140A1BF0010F8AE80700DE
:100DE00000F0D880402385F82B304FF001089AE8B6
:100DF0000700B4463B69ACE803002CF8022BB8F1BD
:100E0000050F4FEA12428CF8002060D9981E424626
:100E100030F8021F002948D10DF1130C072102F010
:100E20000F0E0EF13000392888BF0EF137000F2A5F
:100E30000CF8010901F1FF314FEA121049D808AB53
:100E40005A187E2002F8140C05F11F008446002277
:100E5000914206D01CF801EFBEF1200F02F101090A
:100E600039D107299CBF08AB03EB010C02F1010249
:100E700096BF1CF814CC4FF0200C0131072A00F863
:100E800002C0EED92846FFF7E7FE814600287DD153
:100E900008F10108B8F1640FA9D14FF007094846DD
:100EA00009B0BDE8F08F01348CE74FF0100C01F071
:100EB000010E0EEB4202D30344BF82F4883282F06B
:100EC0002102BCF1010C4FEA5101F0D1A0E74246EA
:100ED000A2E70246A3E74A46BAE729692846A1EBFA
:100EE0004411FFF772FC81460028D8D13046FFF745
:100EF0006EF94FF6FF780190A9693846FFF7E8F9D7
:100F000081460028CBD1EB69019AD7F810E05A73DB
:100F1000E1B24FF00F024FF00D0CDA72DFF8D8A0FB
:100F200018734A1E0CFB02F29876D87684461AF89B
:100F3000019B404518BF3EF8120003F8090003EB7F
:100F4000090B0CF1010C18BF01324FEA10290028DF
:100F500008BF4046BCF10D0F8BF80190E7D140452A
:100F600002D03EF812200AB941F040011970012365
:100F7000FB7100212846FFF73FFD814600288ED1F6
:100F8000013CB9D11AE04FF0060988E7042886D160
:100F900085F82BB01BF0020F1BBF0C340D21012470
:100FA000B4FBF1F418BF013421462846FFF779FD60
:100FB000814600287FF473AF013C8ED1A969384681
:100FC000FFF786F9814600287FF469AF01462022A9
:100FD000E8693FF05BF903CEEB6918605960B278BD
:100FE000318819819A7295F82B30EA6903F0180359
:100FF00013730123FB7152E7D0E80608F8B50446E5
:10100000FFF741F90546002842D16379032B37D118
:10101000277A012F34D104F13C0601464FF40072C7
:1010200030463FF033F9552384F83A32AA2384F846
:101030003B3252234122722184F83C3084F83D3007
:10104000612384F83E3084F83F2084F8222284F81B
:10105000233284F8201284F8211204F50970A16962
:10106000FFF7A2F8616904F50A70FFF79DF8A26A1C
:1010700020680132A2633B46314601F0AEFB257287
:1010800000222068114601F0BDFB003818BF012086
:10109000F8BD2DE9F0470026D0F800A08E758369D1
:1010A00007460C46002B00F09380C36A01336ED1D3
:1010B000F96900234D1E18462E2615F8012F202A07
:1010C00000F101000CD0052A08BFE522092804D14F
:1010D0000B2B9EBFE71801337E72E71801337A723B
:1010E0000B28EAD1E21800205072A27D002A5ED1BE
:1010F000002B53D06FF0080604F109020825361BB7
:10110000B31812F8010B00284BD02E2883B261D0FF
:10111000A3F14100192803D8087B054200D02033F1
:101120001373EDE7B9F1000F05D100F520539BB221
:10113000B3F5006F13D340F2B51140EA094053F004
:10114000D1FBFF28C8F1FF0519D9012D22D904EBE5
:101150000803020A9A75D8750223984400200236C3
:101160008146DAF81030985B0028DBD14546B9F1AA
:10117000000F18BF002525440023AB7598E758B130
:10118000002DF4D004EB080398750123E5E7B14680
:10119000B046E6E70025EAE70546E8E73F23A37502
:1011A0000123234400229A750B7B03B96372CB7A27
:1011B000237201F11C00FEF7EFFF2060CA7D8B7DDA
:1011C00043EA0223E3804A7E0B7E43EA0223A380A4
:1011D000BDE8F0871025A3E72DE9F04F0B78D0F894
:1011E00000B02F2B87B00646884601D05C2B0AD171
:1011F000424613782F2B904602F10102F9D05C2B66
:10120000F7D0002301E0DBF81C30B36098F8003021
:101210001F2B00F22A81802386F82B3000213046D4
:10122000FFF7D3FA07B0BDE8F08FFE2D00F246813C
:101230002AF8153001351EE108F101010591DDF8AC
:10124000148098F800202F2AF6D05C2AF4D0202BA6
:1012500034BF04240024012D2CD1BAF800302E2BE9
:101260002ED100232AF8153006F120029D428CBFB2
:101270002E21202101330B2B02F8011BF6D144F063
:10128000200486F82B403046FFF7E6FC96F82B301A
:10129000002800F0D9800428C4D1990603F0040284
:1012A00040F1CE80002A00F0E080802386F82B30C9
:1012B0000020B7E7022D03D1BAF802302E2BCCD094
:1012C000AAF102028DBB00232AF81530002D00F090
:1012D000F5803AF81320202A194603F10103F8D0CB
:1012E00009B92E2A01D144F00304AAF1020232F80E
:1012F00015302E2B01D0013DF9D14FF020334FF0A6
:10130000000973623362C6F827304F4608233AF863
:1013100011004A1CE8B1202803D02E280DD1954297
:101320000FD044F003041146F1E732F81530202BBA
:1013300001D02E2BC7D1013DC4E7994504D2954277
:1013400033D10B2B2AD101E00B2B22D144F0030423
:101350000B2396F82020E52A04BF052286F82020DA
:10136000082B04BFBF00FFB207F00C030C2B03D007
:1013700007F00303032B01D144F00204A30780D438
:10138000FD0748BF44F01004780748BF44F0080444
:1013900077E7954202D044F00304DAD3BF00FFB2EE
:1013A0002A460B234FF00809BDE77F2813D9CDE962
:1013B000022340F2B51144F00203019353F092FA74
:1013C00010F0800FDDE9022310D03E4900F07F00CD
:1013D000085C019C30B1DFF8F4C01CF8011BE9B1D6
:1013E0008142FAD144F003045F2010E0FF28F0D9D5
:1013F000591E894503D344F00304994693E706EB4D
:101400000901040A81F82040019C09F1010906EB59
:10141000090109F1010981F8200084E7A0F14101E7
:1014200089B2192902D847F00207F0E7A0F161015B
:1014300089B219299EBF203847F0010780B2E6E73C
:10144000002A08BF0520EDE65A073FF5EBAEB37959
:10145000DB0635D533699BF80500C3F308030BF1B0
:101460003C011944FEF7F5FEB0603368CDF81480F6
:10147000D3F810A0002505A8FEF7DBFE421C1DD006
:10148000B0F5803F24BF030C2AF8153083B228BF83
:1014900001351F2B7FF6D3AE2F2B3FF4D0AE5C2B44
:1014A0003FF4CDAE7F2B3FF6C0AE0749184611F88A
:1014B000012B002A3FF4B9AE8242F8D10620B1E6F2
:1014C0000520AFE650E806080CE8060815E806080F
:1014D00000214171FEF750BF2DE9F04305468DB064
:1014E00090461E460C46002900F0BC8003F03F07E2
:1014F0003946FEF741FF002840F0AC80414668467F
:101500000095FFF769FE024620B99DF92B30002BAC
:10151000B8BF062216F01C0F6BD0002A3CD0042A5C
:1015200037D16846FFF742FC024690BB47F00807F8
:10153000DDF81C90A846494618F8050FFEF789FE0D
:10154000064652F0A3FB014609F10E00FEF72CFE01
:10155000079B2022DA72079900224046FEF787FE99
:10156000079B00221A775A779A77DA770123EB7173
:10157000DEB131466846D5F83880FFF7DBF9024620
:1015800038B941462846FEF7A3FE013E6E61024689
:1015900058B10023236028E09DF8063013F0110FA6
:1015A00031D1700758D43107C2D4AB6B079E236288
:1015B000666268793907314648BF47F04007FEF751
:1015C00048FE0146A06006F11C00FEF7E5FD6B89B0
:1015D000A380BA064FF000030646E060256027743A
:1015E0006374E361636110D4002210460DB0BDE85E
:1015F000F083002ACDD19DF80630DA062ED4B60746
:10160000D3D5D807D1D50722C3E70028ECD0EF897E
:1016100060617F02B7420FD30022A161002AB8D1D6
:10162000C6F30803002BDFD02846FEF7C5FDB8B18E
:1016300000EB5620E061D8E72068FFF76CF801283E
:101640000146A6EB070603D9431CE3D10122E4E7D8
:101650000222E2E702469CE708229AE7042298E782
:10166000022296E70922C0E72DE9F04F994685B09E
:1016700000238846C9F8003003A904461746FEF740
:10168000B5FD0646F8B9667CEEB994F810A01AF0DC
:10169000010300937CD0E2686369D21A974228BFA5
:1016A000174687B16269C2F30803002B57D1039B29
:1016B000DB89013B13EA522A15D142B9A0680128FF
:1016C0000AD802266674304605B0BDE8F08FA169DD
:1016D0002068FFF720F8F2E7431C03D10123009EA6
:1016E0006374F0E7A061DDF80CB0A1695846FEF71D
:1016F00063FD0028E5D0B7F5007F0AEB00022DD38B
:10170000BBF80E1001920AEB572088424FEA57258A
:1017100088BFA1EB0A05DBF800002B46414601F02B
:101720004DF80028DAD10399CB795BB1886B019A27
:10173000801AA84206D24FF400723C3108EB4020D8
:101740003EF05EFD6D02D9F800302B44C9F8003040
:1017500063692B447F1BA8446361A2E7E26165696A
:10176000E1690398C5F30805C5F50075BD4228BFBA
:101770003D46FEF7ADFD0028B0D1039963693C31C9
:10178000C3F308032A46194440463EF039FDDAE720
:10179000072698E72DE9F04F9A4685B00023894641
:1017A000CAF8003003A904461746FEF71FFD064697
:1017B00020BB667C16BB237C9A0740F1A980636935
:1017C000FB4200D3DF43AFB16369C3F30802002AD1
:1017D00040F08180039AB2F80E8008F1FF3818EAD1
:1017E00053281ED173B9A06870B901462046FFF78F
:1017F0002DF848B9237C43F040032374304605B0EC
:10180000BDE8F08FA169F1E7012802D102266674D4
:10181000F4E7431C01D10126F9E7A368A06103B9ED
:10182000A0600398E369826B9A4203D1FEF72BFD17
:101830000028F0D1039DA1692846FEF7BDFC0028D1
:10184000E4D0B7F5007F08EB000B36D3E98908EB4D
:10185000572088424FEA5723286888BFA1EB080326
:101860005A464946019300F0B8FF05460028D2D1F8
:10187000DDF80C80019BD8F83810A1EB0B019942E0
:101880000AD24FF4007209EB412108F13C003EF00E
:10189000B7FC019B88F807505D02DAF800306269F6
:1018A0002B44CAF800307F1BE368A94415446561E6
:1018B000AB422CBFE360E56085E76169E36899426C
:1018C00007D32846FEF7DFFC0028A4D1039BC3F80A
:1018D00038B0C4F81CB06569E1690398C5F3080520
:1018E000C5F50075BD4228BF3D46FEF7F1FC002856
:1018F00091D1039863693C30C3F308032A46184426
:1019000049463EF07DFC039B4FF00102DA71C4E7CB
:10191000072673E7F7B501A90546FEF767FC0446FD
:1019200068BB2C7C14F0400429D052F0AFF9296A2E
:1019300007460198FEF7CCFC044600BB6E6AF37ABA
:1019400043F02003F3722868AA6831460530FEF799
:101950008EFCE96806F11C00FEF726FC394606F10C
:101960001600FEF721FC0198B4740123F474C371CE
:10197000FFF744FB2B7C23F0400304462B742046E6
:1019800003B0F0BD13B50446FFF7C4FF28B901A9A1
:101990002046FEF72BFC00B9206002B010BD70B5E8
:1019A0000E468CB000210546FEF7E6FC044660B901
:1019B000314668460095FFF70FFC044690B99DF943
:1019C0002B30002B04DA029BEB6120460CB070BD7B
:1019D0009DF80630DB0609D507996879FEF739FCD2
:1019E000E861F2E7042808BF0524EEE70524ECE7E8
:1019F0002DE9F0470E460021D2B031708146904665
:101A0000FEF7BAFC0546F8B9D9F81C30CDF80090BD
:101A100002934446DDF808A0BAF1000F1AD14445FC
:101A200002BF04F1FF342F233355A11B33461A5D47
:101A300003F8012B5A189045F9D8A8EB0403013498
:101A4000A04538BF01231E4400232846337052B0FE
:101A5000BDE8F08720216846FEF7B7FE00284BD18D
:101A600006994846FEF734FC0746002842D10799FC
:101A700099F80500FEF7EDFB394602906846FEF73F
:101A8000A4FE002838D100216846FFF72DF807464C
:101A9000B0BB079999F80500FEF7DBFB50450AD06B
:101AA00039466846FEF7A8FF0028ECD00546042D0D
:101AB00008BF0225C8E70CA96846FFF7EAFA0DF14E
:101AC000460212F8011B3B4601370029F9D1BC42FE
:101AD00014D331191A4632B9621ED21ADB431C44A0
:101AE0002F23B35496E7013A0CA81044807D01F8E7
:101AF000010DF0E70546A7E70546A5E71125A3E791
:101B00000546D4E72DE9F3410D4601A90446FEF749
:101B10006DFB0646002850D1667C002E4DD1E3684F
:101B2000AB4204D2227C12F0020F08BF1D460022F5
:101B3000636962619DB90020E2686369934282BF74
:101B4000227CE36042F04002C3F3080388BF2274A2
:101B5000002B32D0E369834218BFE0612DE0019A87
:101B6000D7897F02FBB1013B6A1EB3FBF7F1B2FBE1
:101B7000F7F28A4217D37A421340A1696361ED1AE2
:101B80000029D8D0BD42636922D863692B446361C0
:101B9000C5F30803002BCED00198FEF70DFB50B122
:101BA00000EB5520C8E7A16881B92046FEF74EFE3C
:101BB0000128014605D102266674304602B0BDE810
:101BC000F081481C01D10126F6E7A160A161D7E7A9
:101BD0003B446361237C9A07A5EB070806D52046A2
:101BE000FEF734FE054628B90146CEE72068FEF729
:101BF00092FD05466B1CE6D0012DDCD9019B1B6ACA
:101C0000AB42D8D9A56129464546BBE770B5054624
:101C100016460C4621B30021FEF7AEFB68B92560DD
:101C200031462046FFF7D8FAE0B994F92B30002B63
:101C30000BDBA379DB0603D40520002323600EE031
:101C40006879E169FEF705FBA0606B89A38000213C
:101C50002046FEF7BAFD0428EED00028EDD170BD75
:101C60000920FCE70428E7D0E7E713B501A90446FB
:101C7000FEF7BCFA00B9206002B010BD73B50D4686
:101C800001A90446FEF7B2FA20B9014620461DB963
:101C9000FEF79BFD02B070BDFEF726FF10F0FB06BD
:101CA000F8D129462046FFF7F4F931462046FEF7E1
:101CB000A3FE042808BF0020ECE770B50E468CB0E8
:101CC000002104461546FEF757FB0094044670B900
:101CD00031466846FFF780FA044640B99DF92B303B
:101CE000002B07DB1DB129466846FFF7D2F92046D5
:101CF0000CB070BD0624FAE72DE9F84F88460021A4
:101D00000446FEF739FB054640B9D4F820A0A36984
:101D1000AAF10202934204D8C8F800302846BDE870
:101D2000F88F6379012B17D10227064639462046E2
:101D3000FEF7F1FC431C37D0012837D000B901363B
:101D4000236A0137BB42F1D8C8F80060237AA66144
:101D500043F001032372E1E7E16A0746064604F116
:101D60003C0937B9204601F1010BFEF7B1FAF8B989
:101D700059466379022B09EB07000DD119F807309A
:101D8000427853EA022308BF01360237BAF1010A4A
:101D9000C7F30807E5D1D7E7FEF7FEF930F0704347
:101DA00008BF01360437F1E70125CDE70225CBE76F
:101DB0000546C9E7F0B50E4699B002210546FEF783
:101DC000DBFA044688B9314668460095FFF704FA05
:101DD000044650B99DF82B3098063BD4190639D4E7
:101DE0009DF80670FA0703D50724204619B0F0BD08
:101DF00007996879FEF72DFAFB0606460BD468466C
:101E0000FEF702FF04460028EFD1D6B92846FFF7B7
:101E1000F5F80446E9E7EB698342E5D00E902146E8
:101E20000CA80C95FEF7D1FC04460028DDD1014634
:101E30000CA8FEF759FE04460028D5D00428D4D1BA
:101E4000DDE7024631466846FEF774FD0446002889
:101E5000CBD1DBE70624C8E72DE9F0430E4691B06D
:101E600002210546FEF788FA044600286CD1314667
:101E700004A80495FFF7B0F90446002872D004289E
:101E800062D19DF83B1011F020016DD1684600959C
:101E9000FEF7DCFC064600285AD001285AD0431C25
:101EA0005C425C4151F0F2FE0746002C54D13146B1
:101EB0002846FEF777FD044600284DD14FF0203329
:101EC000EB632B64C5F843302E2385F83C30102398
:101ED00085F84730394605F1520005F13C0405F11B
:101EE0000508FEF761F9324621464046FEF7BFF984
:101EF00005F15C031A4651F8040B42F8040B9942B1
:101F0000F9D12E23069A85F85D3040464FF001093D
:101F1000FEF7ADF985F8079004A8FEF747FF0446E1
:101F2000D0B90B9839461630FEF73EF90B99324678
:101F30004046FEF79CF90B9B1022DA72284685F882
:101F40000790FFF75BF80446204611B0BDE8F08328
:101F50000724A7E70224A5E7002231466846FEF7DA
:101F6000E9FCF1E70824EFE70624EDE7F0B50D46BC
:101F7000A1B0022104461746FEF7FEF9002877D1EA
:101F8000294608A80894FFF727F9002870D19DF882
:101F90004B3013F0A00F6DD10F9B6D4603F120065F
:101FA000186859682A4603C20833B3421546F7D168
:101FB00008AE0FCE14AD0FC50FCE0FC596E80F00BB
:101FC00085E80F00394614A8FFF706F948B9169AB4
:101FD0000A9B9A4203D1189A0C9B9A4203D008207C
:101FE00046E0042844D114A8FEF7E0FE00283FD1C3
:101FF0001B990DF10D0301F10D020DF11D0053F8B8
:10200000045B42F8045B8342F9D1188810809B7806
:1020100093709DF80B30DA0658BF43F0200301257A
:10202000CB72E571CB7ADB061BD50A9A169B9A42D6
:1020300017D06079FEF70DF901462046FEF7BCF88F
:102040000146C8B12046FEF743F988B994F85D30DF
:102050002E2B06D1169A04F15C01601DFEF707F9DC
:10206000E57108A8FEF7D0FD10B92046FEF7C6FFBF
:1020700021B0F0BD0620FBE70220F9E7F0B595B0EE
:10208000064601910221FEF777F90446002833D174
:1020900002AF4FF02033029305467B60C7F807304C
:1020A000019B1B781F2B20D89DF80830E52B22D0F0
:1020B0001DB16B1EFA5C202A35D0002108A80896B5
:1020C0000A91FEF782FB0446B0B9012108A8FEF789
:1020D0000BFD98BB0F9A45B33B4603CB1060516094
:1020E00019889B789372118121E001A8FEF7A1F86D
:1020F000B0F5803F03D30624204615B0F0BD52F062
:1021000025FC40F2B51152F0EDFB0028F3D01D4A3A
:1021100012F8013B13B19842FAD1ECE7FF2822D81C
:102120000A2D28D9E7E71D46C2E7E52313700123EE
:10213000F3713046FEF762FF0446DDE70428FBD169
:10214000002DD9D0012108A8FEF7ABFC04460028D9
:10215000D2D1202201460F983EF098F80F9B08221A
:10216000DA720F9AB8E7092DC5D814AB2B44020ACE
:1021700003F8482C013514AB2B44013503F8480C07
:102180008EE700BFDDE806082DE9F04FD0F80080AB
:102190008BB01C46002343710291037901931546CD
:1021A00005210DF11F02404600F02CFB9DF81F3069
:1021B000DA0700F189825E0700F1888208AA03210C
:1021C000404600F01FFB30B9089A531EB3F5004F8C
:1021D00001D21A4201D0012308935DB15C4BA5F5F1
:1021E00000729A4203D913200BB0BDE8F08F6B1E2A
:1021F0002B42F8D1002C00F06B82149BB3F5007FCA
:10220000C0F06682019B002B66D00123002221468C
:10221000404600F0D3FA08B10120E5E794F8FF2129
:1022200094F8FE3143EA02234AF65522934201D044
:102230000E20D9E7019B04EB031303F5D77193F844
:10224000B231002BF4D001F10800FDF7A5FF0746DD
:1022500001F10C00FDF7A0FF0990DDF824A0BAF110
:10226000150FE5D9B5F5813FBDD2029B13F00203EE
:1022700005934FEA5522029B41D003F00703022B3E
:1022800000F03482029BD80740F13082002A3FD10F
:1022900030484FEA1A35012630F8023B0BB1AB4209
:1022A00034D940F6F573BAFBF6F59D429BBF05EBBA
:1022B0004505013502356D088CBF6D0003354FF0C3
:1022C000200305F2FF1504938CBF4FF002094FF075
:1022D00001096D0A01232CE209AA0121404600F000
:1022E00091FA002898D1029B13F0080F099B14BFA4
:1022F00000273F27BB429BD3DB1B0993ADE7D907E0
:10230000C4D470E75200F8E11346FDE17600C3E75C
:102310001646C6E7B9F1020F1ED103994FF6F570C4
:10232000814208D9002A40F0DD817600402E00F27B
:1023300038823246AAE7039940F6F570814213D8F5
:10234000002A7FF475AF7200802A9FD970E700BF22
:1023500000FEFF00F0E80608039940F6F57291428E
:102360003FF666AF4FF001094FF40072002120469E
:1023700005933DF08BFFD74A059B1168216051689A
:102380006160A3731189927A2181C3F30723B9F1A4
:10239000030F4FF00201A272E3734FF000024FF0FF
:1023A0000103237414BF0B461346BAF5803FE27253
:1023B000217366736274A37480F01D8184F813A086
:1023C000CAF3072A84F814A0F82363753F23237601
:1023D0004FF0000AFF2384F819A0A37684F81BA00D
:1023E000394604F11C00FDF7DFFEB9F1030F40F0A0
:1023F000088151F04BFC014604F14300FDF7D4FE87
:10240000294604F12400FDF7CFFE022384F82C3086
:10241000012384F83030062384F83230802384F896
:102420004030292384F84230AB4B84F82DA084F847
:102430002EA084F82FA084F831A084F833A004F1F2
:10244000470203F1100153F8040B42F8040B8B42CE
:10245000F9D119889B7893704FF05503118084F857
:10246000FE316FF0550384F8FF313A4601232146CF
:10247000404600F0B2F9824600287FF4CDAEB9F1B3
:10248000030F3ED10123BA1D2146404600F0A5F9B5
:102490004FF40072514620463DF0F8FE522323705F
:1024A00063706123A37084F8E731039B412272219A
:1024B000E27084F8E41184F8E51184F8E621591EED
:1024C00004F5F470FDF770FE022384F8EC314FF050
:1024D000550384F8FE316FF0550384F8FF31FA1D7F
:1024E0000123214684F8EDA184F8EEA184F8EFA140
:1024F000404600F072F90123FA182146404600F0E8
:102500006CF9149B23F4FF7222F001020021204693
:102510003DF0BCFEB9F1030F40F09080F82323702A
:10252000FF236370A370E37023716371A371E37180
:1025300023726372A3720F23E372149B5B0A0393EB
:10254000039BAB4228BF2B4621465A4640469A463B
:1025500000F043F9014600287FF45EAE4FF40072AC
:1025600020463DF093FEB5EB0A05D344E8D1049B29
:10257000B9F1030F18BF1E46039BB34228BF334671
:102580005A46214640461D4600F027F900287FF4B0
:1025900043AE761BAB44EFD1B9F1030F58D0099B82
:1025A000B3F5803F56D2B9F1020F0CBF04250125C7
:1025B000019B002B50D0002201232146404600F011
:1025C000FDF8024600287FF427AE019B04EB0313BD
:1025D00083F8B25101232146404600F0FEF800285E
:1025E0007FF41AAE00221146404600F00BF9003885
:1025F00018BF0120F8E5514604F12000FDF7D4FD95
:10260000E2E651F043FB014604F12700FDF7CCFD63
:10261000C5F30723E375802384F82430292384F845
:1026200026302E4BA57504F12B0203F1100153F84F
:10263000040B42F8040B8B42F9D10AE7B9F1010F00
:102640002749204618BF6FF00701FDF7ADFD74E77D
:102650000C25ADE70625ABE7029B1B07C2D4019909
:102660004FF4007220463DF011FE5523099A84F87C
:10267000FE31AA2384F8FF31019B84F8BE3184F82F
:10268000C1313A4443F6C163B2FBF3F2FE2384F84E
:10269000C331930843F03F03012684F8C43184F822
:1026A000C521394604F5E37084F8BF6184F8C06140
:1026B00084F8C251FDF778FD099904F5E570FDF73E
:1026C00073FD019A334686E703208DE50A208BE5EA
:1026D000112089E51CE8060828E806083CE80608F9
:1026E000F8FFFF00059B002B3FF4A2AD002A7FF40A
:1026F0000BAE30484FEA5A45012230F8023B1BB17D
:10270000AB427FF6FFAD0023BAFBF2F02A4E850004
:10271000A0F57F40F63805F20725B0424FEA55256F
:102720003FF686AD16461A46002304934FF0030980
:1027300020230498DDF820E007EB030B05EB000CE9
:10274000DC440EF1FF306044CEF1000E00EA0E00D2
:10275000A0EB0C00B9F1030F06BF1B1883442D1822
:10276000C7EB06108444E245FFF462AD0498AAEB7F
:102770000000C01AB9F1030FA0EB0500B0FBF6F0A2
:1027800003907FF4C7AD03994FF6F57081423FF691
:10279000EBAD002A7FF44CAD012E7FF649AD7208F7
:1027A000A4E7059B002BA4D1802E3FF641AD324615
:1027B00077E500BFFEE80608FFFFFE0F10B50C46E8
:1027C00011461A4638B1234604303CF075FB0038F8
:1027D00018BF012010BD0420FCE710B50C461146BF
:1027E0001A4650B1234604303CF0A8FB10F11E0FEE
:1027F00005D0003818BF012010BD0420FCE70220DE
:10280000FAE7000070B50D4614460646002833D09E
:10281000244A01F00703D15C00292FD000220430A4
:102820003CF0D8FB062D27D8DFE805F008050A168E
:102830002619190006202AF0B5FD2060002070BD81
:10284000062805D14FF4007323802388B360F5E791
:102850002AF0A8FD2080F8E701232360EEE7062890
:1028600001D0430806D1336A002B0CBF0423002398
:102870002370E3E70123FBE70420E0E7062DFBD804
:1028800001A353F825F000BF3D28000835280008B3
:1028900045280008592800087928000867280008FA
:1028A0006728000838350608086833F054B9000076
:1028B00037B51D46043001AB1446FEF76BFF38B147
:1028C000064B1B5C2B604FF0FF34204603B030BD3D
:1028D000019BA342F9D01C23F4E700BF783506081A
:1028E00013B51C46043001ABFEF7BEFE30B1044BFD
:1028F0001B5C23604FF0FF3002B010BD0198FBE776
:10290000783506082DE9F843814650680E46904612
:1029100030F076FC2E4A2F490138002410F8013F90
:10292000D3B92C201DF0CCFB0746054647F8046BB5
:10293000D8F8000030F064FCE3B20246394609F1F1
:102940004400FEF7C9FD0646C0B328461DF0D2FB81
:10295000214B985D29F00CFF782BDFD8712B08D81C
:10296000612B24D0622B25D02B2BD7D144F003042C
:10297000D4E7723B062BD1D801A555F823F000BF50
:102980009D2900081D290008B92900081D290008F3
:102990001D290008A3290008A929000844F0010402
:1029A000BCE744F00A04B9E744F00604B6E744F093
:1029B0001204B3E70E46B1E71646AFE7E30603D5C8
:1029C00029693846FFF79EF82846BDE8F88300BF1E
:1029D000C83506088C3506087835060830B587B046
:1029E000044603AD084611461A46064B009301956E
:1029F00003232AF0D5F92A4621460020FFF782FF5B
:102A000007B030BD603506081FB50623CDE90112B9
:102A10000349039301AAFFF775FF05B05DF804FBB6
:102A2000C835060813B50446084601912AF02EFC65
:102A3000019B04490246204602B0BDE8104000F068
:102A4000BBBF00BF40350608022970B504461546D5
:102A50001E4613D15368012B0AD0022B0CD01BB990
:102A60001168201DFFF74EF8A3692B60002070BD90
:102A700081692B681944F4E70169FAE701290AD151
:102A80000430FEF747FF0028F0D0084B1B5C336092
:102A90004FF0FF30EBE7042906D14368002BE5D067
:102AA0000430FEF76FFFEEE71623F0E778350608EF
:102AB0002DE9F74F06299DF8305010D8012905D986
:102AC0003F2300F8013B0023037001E00029FAD105
:102AD000012994BF0020012003B0BDE8F08F10EE63
:102AE000104A002C044622DAB4EE400AF1EE10FA45
:102AF0001DD62D2504F8015BB1EE400A9FEDC27A88
:102B0000F0EEC07AF4EE477AF1EE10FA02F0200E01
:102B100012DD8EF0490323708EF046058EF04E03D1
:102B20006370E11CA57000230B70081AD4E7002D18
:102B3000E4D004F8015BE1E7B4EE400AF1EE10FAEC
:102B400008D74EF04E038EF0410523706570E11CEE
:102B5000A370E8E7002B42F02002B8BF0623672AE3
:102B600002D1002B08BF012310EE106A251A491B61
:102B7000002E01F1FF3547D1662A37D15E1CAE42E7
:102B8000A8BFCB1E00275D1C6621BC463E466529BA
:102B900023EAE37840F0098108F10105002301935D
:102BA0004FF02E0BB2EE047A019B9D4200F306819A
:102BB000662A40F03381AE4240F3848197B10A2106
:102BC00096FBF1F301FB136693FBF1F201FB12326A
:102BD0004EF0450E3032303684F800E06770A27057
:102BE000E670043400232370201A75E75E1DAE42A0
:102BF000A8BFCB1F652A11464FF0000540F0CF80DB
:102C00002B27AC462E46C2E7B6F17E5F6FD2DFEDD2
:102C10007F7ADFF80082DFF800A2B4EEE70AF1EE77
:102C200010FA4FF00007ACBF4FF031094FF03009F8
:102C30004FF0200C3E46B8EC017AB4EEC07AF1EECB
:102C400010FAC4BF0AEB070B9BED007A07F10407EB
:102C5000C4BF664420EE070A182F4FEA6C0CEAD175
:102C600010EE107AB7F17E5F27D2B4EEE70AF1EEEC
:102C700010FA1DDB002E14BF2D272B27B7EE000AFC
:102C8000662A03D0672A28D1042E26DC672A04BFCF
:102C900006F1FF37DB195F1CAF42A8BFCB1E84F8DB
:102CA000009063B901341D461F464FF0FF3C58E0C9
:102CB000F2EE047A20EE270A01362D27E0E72E21D6
:102CC00061701D4602343021013E6AD00DB92F4695
:102CD000EBE704F8011B013DF6E78D1F9D4202DC86
:102CE000672A60D0CB1F11460025AC464FE700276E
:102CF000DFF82481DFF81C914FF0200C3E46F8EC01
:102D0000017AF4EEC07AF1EE10FA9CBF09EB070AE3
:102D1000DAED007A07F104079CBF664420EE270A2B
:102D2000182F4FEA6C0CEAD1FDEEC07A17EE907ABC
:102D3000092FC2BFDFED367A013620EE270A662A58
:102D400011D1AE4217DA99190131A94205DBAD1B49
:102D5000012DA5F1020308BF0023F5180135B44683
:102D60000027662113E7652A05D0672A0CD0114693
:102D700000252B27B9E78D1F9D4200DCCB1F0025C6
:102D80002B27AC46652102E71F1DAF4200DB8B1FDE
:102D90009E4201DB6721EBE7711C5B1ADDE72F46E2
:102DA0002FE7374681E72B469DE767297FF4F6AE8C
:102DB000002BDABF0125A8464546EFE6FDEEC07AB6
:102DC00004F1010A17EE903A002BA8BF03F1300975
:102DD000019BACBF5FFA89F94FF030099C4584F83C
:102DE000009006D1B8F1000F03D004F1020A84F874
:102DF00001B0F8EEE77A019B30EE670A013320EE6E
:102E0000070A01935446CFE6FFFF7F7FF8FF7F3F1D
:102E1000CDCCCC3D94DE0508ACDE0508F1EE047A9D
:102E2000B4EEE70AF1EE10FA24DB631E4FF030092E
:102E30001D782E2D03F1FF3C2ED0A5F1300ABAF1FA
:102E4000090F2BD901331D78302D13D193F801C010
:102E5000BCF12E0F2FD166292DD02D2F83F800C065
:102E60005D7026D1013E08BF2B2721468B4224D31B
:102E700031211970672A7FF4A1AEB8F1000F3FF439
:102E80009DAE23461C46013B14F8012C302AF9D094
:102E90002E2A08BF1C4691E66346C9E7392D02D0A9
:102EA00001351D70CFE798428CF80190F4D10346AC
:102EB000C9E70136D9E70134D7E711F8015C01F819
:102EC0000159D3E7F1EE047AB4EEE70AF1EE10FA15
:102ED000ABDA73E608B5044631B1054B8A6B036083
:102EE000096800232CF07AFA20461DF0B5F800BFDF
:102EF000F8EE05082DE9FF471E460192451812B16C
:102F0000023A222A34D80446AC42274639D214F871
:102F1000010B1EF067F980460028F5D13B782B2B7A
:102F200029D12746E91B384601AA27F03CFF074470
:102F3000B9460024A9454B4626D3B8F1000F00D06E
:102F40006442640044F00104BB4209D01F46AF4212
:102F50003B4641D2187801371EF044F90028F6D1DB
:102F60002049019A20482CF0FDF93146FFF7B2FFC5
:102F70001E4829F015FA2D2B04BF27464FF00108F3
:102F8000D0E74FF00008CDE719F8012BA2F1300A85
:102F9000BAF1090F09D95F2ACCD042F02002A2F180
:102FA00061011929C9D8A2F1570A01995145C4D91B
:102FB000204636F049FE28B9019B03FB04A494EA9D
:102FC0004403B7D5019B03974246E91B03A82DF0A4
:102FD000D5FB039B0446B7E7C2D1204604B0BDE849
:102FE000F08700BFD9DE0508E8EF0508C4DE050854
:102FF0002DE9F04F2DED028B83B00446DDF83880CB
:10300000019391464618B442254680F031812878D4
:103010001EF0E8F8013407460028F4D12B782B2B5A
:1030200009D125468246B4420CD30023DFED938AB2
:103030001F4618468BE02D2B03D125464FF0010A81
:10304000F1E782462B7843F02003692B32D1AB1C89
:103050009E4240F205816B7843F020036E2B40F0D6
:10306000FF80AB7843F02003662B40F0F980EB1D26
:103070009E4205F103041AD9EB7843F02003692B33
:1030800015D12B7943F020036E2B10D16B7943F0CF
:103090002003692B0BD1AB7943F02003742B06D1AD
:1030A000EB7943F02003792B01D105F108049FED62
:1030B000748A14E06E2B2AD1AB1C9E4240F2D08061
:1030C0006B7843F02003612B40F0CA80AB7843F06B
:1030D00020036E2B40F0C4809FED6A8AEC1CBAF18D
:1030E000000F01D0B1EE488AA54209D0B442234670
:1030F00080F09880187801341EF074F80028F5D11B
:10310000614962482CF0A4F84146FFF7E3FE002332
:10311000DFED5A8A9FED5E7A0093AC461846194659
:10312000F2EE046A644614F801EBAEF1300BBBF129
:10313000090F38D8022922D1564A904202DC0A22CD
:1031400002FB00B0A6425ED8009A02B1404203449E
:1031500013F1250FBEBFDFED507A253368EEA78A45
:1031600013F1090F53D35B4200EE903AB2EE040A1A
:10317000F8EEE00A3EF0EAF888EE808AAFE7F4EE77
:10318000C78AF1EE10FA0BD507EE90BAF8EEE77A9F
:103190000129E8EEA67AF0EE678A31D1013BD1E74A
:1031A00029B90133CEE721B9BEF12E0F03D1012198
:1031B000C8E7022917D04EF0200BBBF1650F12D1E2
:1031C000A64258D99CF801102B2905D10CF1020414
:1031D000B44295D00221B5E72D2913D101220CF17B
:1031E00002040092F4E7B9F1000F04D04EF0200B76
:1031F000BBF16A0F09D0BEF15F0FA3D06446A3E70D
:1032000000219FE70221A4468CE74F469CE707EE8A
:10321000903AB2EE040AF8EEE70A3EF097F828EE8C
:10322000808A5CE77FF46CAF57B19FED140AF0EE33
:10323000480A03B0BDEC028BBDE8F04F2BF0BCB8E0
:10324000019B23B1DFED0D0AB0EE480AF1E7B0EEC5
:10325000480A03B0BDEC028BBDE8F04F2CF0DCB99E
:10326000BAF1000F3FF44CAF9FED048A2C4639E7CA
:103270004FF0000AD9E63FF443AF65E700000000D5
:103280000000807F0000C07FE5DE0508E8EF05084C
:10329000EC78AD6064666606EA1C080208461146D2
:1032A00049F04CBA37B50546084601913DF026F87D
:1032B000044620B102466B68019928689847204669
:1032C00003B030BD2DE9F74F89469DF83010174601
:1032D0000D9A11F0DF0F0646A2EB07023DD0302910
:1032E00025490CA813BF804688464FF0100A4FF0BE
:1032F000010A13F0800535D002EBD2746510A2EB01
:103300006404002D35DDAB46DA45524673683068FB
:10331000A8BF5A46414601929847019AABEB020B6F
:10332000BBF1000FF0DC2FB1736830683A464946B4
:1033300098473D44002C0CDD2544A2455746A8BFC4
:103340002746736830683A464146E41B9847002C8C
:10335000F3DC284603B0BDE8F08FDFF820804FF0A3
:10336000100AC6E713F0010401D11546C9E7144657
:10337000D9E70025D7E700BF71CF050860CF050862
:103380002DE9F04389B006460020119D9DF8488044
:10339000139F8DF80F000AB381421ADA2D228DF89F
:1033A0000F204942109A08ACA2F10A000DF1100951
:1033B000B1FBF3FC03FB1C12092A8CBF121830323C
:1033C00004F8012D4C458E4661460ED07345EFD969
:1033D0000BE0A80727D52B228DF80F200029E1D17B
:1033E00030238DF81F300DF11F0415F040099DF8B2
:1033F0000F301CD023B30122CDE900822B460DF102
:103400000F013046FFF75EFF013F814608AACDE974
:1034100000872B46121B21463046FFF753FF4844D6
:1034200009B0BDE8F0836A07D8D52022D4E7002B85
:10343000ECD004AA9442E9D904F8013C013CE5E748
:103440009946E3E72DE9F04F93B081461D46C80742
:103450009DF874301C9E0693DDE91E7A0C4690465A
:103460000BD4A10703D12268794B9A4205D020469C
:1034700029F098FF400040F0010416F0810306D1C6
:10348000069A302A03D15745B8BF57469A46204678
:103490002DF086F800280DF1280B18DBB20712D5A5
:1034A0002B238DF828300DF12902F006EDB21DD541
:1034B000B8F1020F0DD11346302103F8021B691C2D
:1034C00051701A4612E0730701D52023E9E75A46E6
:1034D000EBE7B8F1080F60D1B1054FF0300313707E
:1034E00045BF05F10E03537001320232A2EB0B030C
:1034F000002116F0200F117005930EAA0CBF0B4689
:103500002C23BAF1010F0B92C8BF46F040061022DF
:10351000CDE90C2116F04002CDE902538DF82710B9
:10352000079244D0CDE9008123460DAA0CA90BA82F
:103530002CF016FF03782D2B804606D18DF827300E
:103540000D9B013B00F101080D93BAF1010F3CDD29
:103550000D9D079B5545B8BF55462BB19DF82730AB
:1035600003B10135059B1D44AF422BDD16F001036D
:10357000A7EB050527D12C461D4626F001064CB1C8
:10358000202300930023019432491A464846FFF74E
:1035900099FE04463023069319E0B8F1100FA5D127
:1035A0001346302103F8021B05F1170188E70AAB27
:1035B000CDE900830DAA23460CA90BA82CF0D0FE60
:1035C0008046C2E700250024D7E700252C46079B4C
:1035D000DBB19DF8273053B100230122CDE9003241
:1035E0000DF127014846FFF76DFE013F0444059B9E
:1035F0005BB100230122CDE900325946059A4846C5
:10360000FFF760FE059B0444FF1A069B0093BAF186
:10361000010FC8BF57460D9A0197334641464846A9
:10362000FFF750FE04444DB12023009300230949C5
:1036300001951A464846FFF745FE04440B980EAB29
:10364000984201D01CF056FD204613B0BDE8F08F23
:1036500038F50508B38F06082DE9F04316468BB000
:10366000B207DDF84890074698463DD416F0040F9F
:103670000CBF0023202300930A46139B202102A89D
:10368000FFF716FAF30504460DD5431C1F2B0AD885
:103690000AAA1444252204F8202C0AAA1A4400215C
:1036A00002F8201C1C4616F040051FD09DF808307B
:1036B0002F2B4FF000031BD8012202A9CDE90032C5
:1036C0003846FFF7FFFD09F1FF390546013C0DF1D2
:1036D0000901CDE90089334622463846FFF7F2FD5D
:1036E00028440BB0BDE8F0832B23C4E702A9F0E720
:1036F00002A91D46EDE700002DE9F04F824689B092
:10370000144600260B461D4613F8012B82B9A94228
:1037100011D30B78002B00F04681013120234FF0AC
:1037200000080A4612F8015B7DB94FF00A0C2AE046
:10373000252AE8D1EBE76F1ADAF80430DAF800004E
:103740003A4698473E442946E3E72D2D03D148F0F9
:1037500001081146E5E72B2D02D148F00208F8E7F1
:10376000202D02D148F00408F3E7212D02D148F0C2
:103770000808EEE7302D22D148F040082B46E8E754
:103780000CFB0525303D0F4611F8012BA2F130004E
:103790000928F5D92E2A42D17A782A2A11D00A4648
:1037A0004FF00A0C0021174612F801BBABF13000B4
:1037B000092809D80CFB01BBABF13001F3E7002568
:1037C000B3E754F8041B023721EAE17B3A786C2A0C
:1037D00008BF013797F80090B9F1000F00F0E380BF
:1037E000B9F1780F6BD8B9F1570F1BD8B9F1470F62
:1037F00062D8B9F1440F62D9073424F00704F4E821
:103800000201049354F062FBCDE9005B00EE100A64
:10381000049B424649465046FFF71EFF63E04FF0C7
:10382000FF3BD3E7A9F15802202A48D801A151F85B
:1038300022F000BF75390008BF380008BF38000803
:10384000BF380008BF380008BF380008BF3800087C
:10385000BF380008BF380008BF380008D13800085A
:10386000F338000859390008F9370008F93700081B
:10387000F9370008BF380008BF380008BF38000813
:10388000BF380008BF380008BF380008BF3800083C
:10389000BF3800089739000807390008BF3800080A
:1038A00031390008BF38000875390008BF380008F2
:1038B000BF38000875390008B9F1500F6BD0DAF83D
:1038C0000430DAF8000001223946984701360BE04F
:1038D00054F8042BCDE9003543463AB1344904226B
:1038E0005046FFF7EFFC0644791C0BE731490522EF
:1038F000F6E754F8042B8DF81C20CDE900350122A1
:10390000434607A9ECE707A954F8040B04931DF0FC
:103910003CFABBF1FF3F049B014604D0079A934554
:1039200038BFCDF81CB0CDE90035079A4346D7E73C
:1039300054F8041B0593084604913CF0DFFCBBF1EE
:10394000FF3FDDE90413024602D0584528BF5A461E
:10395000CDE900354346C3E7CDE902356123009345
:10396000CDF804800A23012254F8041B5046FFF7C7
:1039700007FDB8E729F00F0209F101010F3A01F044
:103980000601D2B2CDE90235CDF804800092C1F132
:1039900010030022E8E7CDE9023561230093CDF85A
:1039A00004801023F5E7304609B0BDE8F08F00BF72
:1039B0004CCF050851CF05080EB403B503AA52F841
:1039C000041B0192FFF798FE02B05DF804EB03B010
:0439D000704700003C
:020000040802F0
:10000000034B1B685B681A69026018610020704727
:10001000E8620020034B1B685B681A6912681A616A
:10002000704700BFE8620020C460056146618761D7
:10003000C0F81C80C0F82090C0F824A0C0F828B0F8
:10004000C0F82CD080ED0C8B80ED0E9B80ED10ABBA
:10005000C0F808E0FFF7D4BF08B5114B1B6859681A
:100060000B690BB92BF044FA1A6858600A611846FC
:10007000C468056946698769D0F81C80D0F820906B
:10008000D0F824A0D0F828B0D0F82CD090ED0C8B6C
:1000900090ED0E9B90ED10ABD0F808E0012070477A
:1000A000E862002010B50021044600F0B9FA18B942
:1000B00014B120460CF060F910BD002100F0B0BA78
:1000C00010B50121044600F0ABFA18B914B120466E
:1000D0000CF052F910BDFFF7E5BF10B501220C4638
:1000E00000F0B2FB18B914B120460CF045F910BD70
:1000F00000F0AABB00F06ABB2DE9F0432A4C0025B2
:100100000326D4F8F4710021013143189A0803F052
:100110000303BA5C5B0042FA03F303F00303022B10
:10012000F2D0D4F8003209018A0803EB001089B339
:1001300000EB820103681A0729D1D4F800229A4201
:1001400025D89A1AC2F301174FEA470ED4F8047261
:100150009F424FEA921C4FEA121218D9D4F8F48148
:1001600018F80C9049FA0EF707F00307012F0ED18B
:1001700006FA0EF304EB450E3F2D43EA090308F897
:100180000C309ABF0135AEF80C22C4F80872043066
:100190008842CFD12DB1013D04EB4503B3F80C02E9
:1001A000AFE7BDE8F08300BF205C0020F0B4194E3B
:1001B000D6E97F43C01AC109C0F30215635C01226E
:1001C000AA4023EA02036354D6F89822830904095B
:1001D000B2EB901FD6F8F40188BFC6F89832C15C24
:1001E000A50804F0030303275B0007FA03F321EAE1
:1001F000030343550134D6F8F401A50804F00303C2
:10020000415D5A0041FA02F202F00302022AEBD0E9
:10021000F0BC7047205C002021F00F0370B5144A39
:10022000144D1C1AE400A2FB0424640A0219A3EB77
:100230008416C5F8FC2100212246C5E98063C5E982
:100240007D0420F023F8A2000732D2080021D5F85F
:10025000FC0120F01BF800234FF480314FF0FF32F7
:10026000C5E9A432C5F88C12C5F8983270BD00BF3C
:10027000F32C23FA205C0020034AB2F88C320133BD
:10028000A2F88C32704700BF205C0020034AB2F80D
:100290008C32013BA2F88C32704700BF205C0020FA
:1002A000034BB3F88C02003818BF0120704700BF21
:1002B000205C0020F8B51D4CB4F88C3200220133CC
:1002C000A4F88C32C4F89022C4F80822251D04F545
:1002D000E876032755F8042F13071AD1D4F8000243
:1002E000824216D3D4F80412101AC0F301138A42C2
:1002F0004FEA901C4FEA43034FEA101009D2D4F89A
:10030000F41111F80CE04EFA03F202F00302012A94
:1003100002D0AE42DED1F8BD07FA03F343EA0E0382
:1003200001F80C30FFF7E8FEF3E700BF205C002087
:1003300081B3F8B5041F184E04EB8105032754F868
:10034000043F1A071AD1D6F80002984216D8D6F8F8
:100350000412181AC0F3011299424FEA901C4FEA96
:1003600042024FEA101009D9D6F8F41111F80CE046
:100370004EFA02F303F00303012B02D0A542DED1B3
:10038000F8BD07FA02F242EA0E0201F80C20FFF76C
:10039000B3FEF3E7704700BF205C00202DE9F04F6B
:1003A0005A4CD4F8083285B0002B00F0AB80D4F85A
:1003B000F83100269A00C4F80862002A43D00025CC
:1003C000D4F8F411AB08CB5C05F0030149000B41F4
:1003D00003F00303032B41D001359542F0D3D4F849
:1003E0000832002BE7D172B34FF0000E76464FF083
:1003F000030A4FF001094FF0020804E0012B4BD033
:10040000013696421FD2D4F8F4C1B70806F00305AE
:100410001CF807106D0041FA05F303F00303022BEB
:100420000CEB96002AD0032BE8D108FA05F521EA57
:1004300005010CF80710D4F8F83101369A009642FD
:100440004FF0000EDFD3B4F88C320022013BA4F849
:100450008C32C4F8982205B0BDE8F08F2846FFF72B
:100460004BFED4F8F8310135B5EB830F4FEA830228
:10047000A6D3D4F80832002B9DD1B4E7BEF1000F0B
